:020000000140BD
:020003000157A3
:05000B0002005101405C
:2000400075811AD2AFD2A9D28C12005A12001B80FB438CDC050832050832740075F000F52B
:200060000985F00A740075F000F51585F016748075F025C0E0C0F0120ACA15811581120B8D
:200080001979FA7A0CE98AF0C0E0C0F0120AED158115811201ED1201881202001207671225
:2000A000022A1202B41203A512050D12058C120787120874020096227F09120BA8740078AA
:2000C000FC120B9CF6740075F00008F608A6F078FC120B9CE6120BCE7B0A120BC5120C9BE2
:2000E00045F0700302013A801678FD120B9CE60886F0120C5818F608A6F0120C6180D0748E
:200100001175F000C0E0C0F0120B0115811581120B19C0E0C0F0120B291581158178FC1251
:200120000B9CF608E60886F079F6120BA1120BBE78FC120B9CE6F70200E978FD120B9CE6A5
:200140000886F079F6120BA1120BBE7400F778FD120B9CE60886F07B007C00120C9245F040
:20016000700302016D74FF75F0FF02018379F6120BA1E98AF0C0E0C0F0120B4915811581CD
:200180000201837FF7020BB7E598540175F0007B007C00120C9B45F070030201B0120B1927
:2001A000C0E0C0F0120B2915811581F5100201B474FFF51022E598540175F0007B007C00F9
:2001C000120C9B45F070030201D2120B3EF5100201D674FFF51022792D7A0DE98AF0C0E0E6
:2001E000C0F0120AED158115811201ED2279297A0DE98AF0C0E0C0F0120AED1581158122C5
:20020000E510120BCE7B0A120BC5120C9245F0700302022979FA7A0CE98AF0C0E0C0F01254
:200220000AED158115811201ED22E510120BCE7B65120BC5120C9245F070030202B3D2B343
:20024000D2B4C2B5D2B2C2B6C2B71208E3C2B3746475F000C0E0C0F0120B7F15811581E580
:200260000E75F0007B557C00120C9245F0700302027AC2A700D2A702028EC2A7740A75F029
:2002800000C0E0C0F0120B7F15811581D2A7740A75F000C0E0C0F0120B7F15811581D2B34D
:2002A000746475F000C0E0C0F0120B7F158115811201D722E510120BCE7B77120BC5120C0B
:2002C0009245F070030203A4D2B3C2B4D2B5D2B2D2B6D2B7D2A71208E3E50F75F0007BFFDB
:2002E0007C00120C9245F070030202EEC2B3746475F000C0E0C0F0120B7F158115817400FA
:2003000075F000F51385F014740075F000F50985F00AE509850AF0AB15AC16120CA545F0AA
:20032000700302038F8012E509850AF0120C58F50985F00A120C6180D9741175F000C0E062
:20034000C0F0120B0115811581E509850AF0F51185F012851190E5124480F5A01208E31224
:200360000B3EF580741375F000C0E0C0F0120B0115811581E5138514F02580C5F03400C565
:20038000F0F51385F0141208C012092C020327D2B3746475F000C0E0C0F0120B7F15811536
:2003A000811201D72205810581E510120BCE7B72120BC5120C9245F0700302045B74007553
:2003C000F000F51385F014D2B3D2A7C2B4C2B5C2B2D2B6D2B77431F50D740075F00078FD37
:2003E000120B9CF608A6F078FD120B9CE60886F0AB15AC16120CA545F0700302045880163D
:2004000078FD120B9CE60886F0120C5818F608A6F0120C6180D178FD120B9CE60886F0F5D1
:200420001185F012851190E5124480F5A07580FFE5138514F02580C5F03400C5F0F5138569
:20044000F014E58075F000C0E0C0F0120460158115811204870204001201D7158115812201
:2004600078FB120B9CE6F50BE50B75F0007B047C00120C47F50B1204AA78FB120B9CE6548F
:200480000FF50B1204AA221201B57B137C00120C9245F070030204A91201B57B117C0012B0
:2004A0000C9B45F0600302049822E50B75F0007B097C00120CB545F070030204D2E50B2481
:2004C0003775F000C0E0C0F0120B01158115810204E4E50B243075F000C0E0C0F0120B01E5
:2004E0001581158122E58075F0007BFF7C00120C9B45F0700302050C7430F50DE519851A37
:20050000F0120C58F51985F01A120C6122E510120BCE7B6C120BC5120C9245F0700302052F
:200520008BC2B3D2A7D2B4D2B5D2B2D2B6D2B7746475F000C0E0C0F0120B7F158115811239
:2005400008C0740575F000C0E0C0F0120B7F15811581C2B6C2B71208E31208C0740575F037
:2005600000C0E0C0F0120B7F15811581C2B5D2B6C2B71208E31208C0740575F000C0E0C0D6
:20058000F0120B7F158115811201D722E510120BCE7B63120BC5120C9245F070030205D0C8
:2005A000743275F00DC0E0C0F0E5138514F0120C6B2401C5F03400C5F0C0E0C0F0740275CB
:2005C000F00012097515811581158115811201D722D2B3D2A7C2B4C2B5C2B2C2B6C2B77473
:2005E0003175F000F51185F012851190E5124480F5A01208E374FFF580E580F50EE50E75AD
:20060000F0007BFF7C00120C9245F07003020630740075F001F51185F012851190E512449C
:2006200080F5A01208E374FFF580E580F50ED2B5E5118512F0120C58F51185F012120C61D2
:20064000851190E5124480F5A01208E374FFF580E580F50F221205D1E50E75F0009006BE20
:20066000020BD7740075F010F51785F0180206DE740075F010F51785F0180206DE740075DD
:20068000F020F51785F0180206DE740075F020F51785F0180206DE740075F050F51785F0A9
:2006A000180206DE740075F050F51785F0180206DE740075F000F51785F0180206DEB10685
:2006C000FF00A4066500970655008A0662007D06520070066100630651000000DE0674006A
:2006E00075F000F51385F014740075F000F51985F01AD2B3D2A7C2B4C2B5C2B2D2B6D2B71E
:200700007431F50D740075F000F50985F00AE509850AF0AB17AC18120CA545F07003020775
:20072000668012E509850AF0120C58F50985F00A120C6180D9E509850AF0F51185F012850A
:200740001190E5124480F5A0C2B574FFF580E5138514F02580C5F03400C5F0F51385F014F4
:200760001204E502072322E510120BCE7B73120BC5120C9245F070030207861200B8F515C5
:2007800085F0161201D722E510120BCE7B67120BC5120C9245F07003020873120655E50EE9
:2007A00075F0007BFF7C00120C9B45F07003020860744275F00DC0E0C0F0E50E75F000C083
:2007C000E0C0F0740275F0001209751581158115811581E50F75F0007BFF7C00120C924582
:2007E000F070030207F6745175F00DC0E0C0F0120AED15811581E50F75F0007B057C001274
:200800000C9245F07003020819745675F00DC0E0C0F0120AED15811581745A75F00DC0E0CE
:20082000C0F0E519851AF0C0E0C0F0740275F0001209751581158115811581746E75F00D14
:20084000C0E0C0F0E5158516F0C0E0C0F0740275F000120975158115811581158102087036
:20086000748175F00DC0E0C0F0120AED158115811201D722E510120BCE7B70120BC5120CB5
:200880009245F070030208BF120655749375F00DC0E0C0F0E50E75F000C0E0C0F0E51985F4
:2008A0001AF0C0E0C0F0E5158516F0C0E0C0F0740475F0001209757FF8120BA81201D72254
:2008C000E50E75F0007B557C00120C9245F070030208DBC2A700D2A70208E2C2A700000000
:2008E000D2A72205810581740075F00078FD120B9CF608A6F078FD120B9CE60886F07B01A8
:200900007C00120C7245F07003020927801678FD120B9CE60886F0120C5818F608A6F01295
:200920000C6180D102090E158115812205810581740075F00078FD120B9CF608A6F078FD76
:20094000120B9CE60886F07B147C00120C7245F07003020970801678FD120B9CE60886F094
:20096000120C5818F608A6F0120C6180D1020957158115812223F42581F8868208868308FF
:20098000E4FEFF93700122B42555A3E493B42D06430780A3E493B4300343074024D0B40A1A
:2009A00000500CCE75F00AA42EFEA3E49380EDE493B46413E60886F030F708430720120C8A
:2009C00068A6F018F68003B4750543070A801CB478054307108014B46F0B430708800C122D
:2009E0000B07A3809BB462624307027A00C004C005C006C007AB0753031F7C00E60886F0CC
:200A0000120C14A6F018F6EDD007D006D005D0042430B43A0040022407C0E00AE645F070D9
:200A2000CCA902EF30E506742D120B070A120AABD0E0120B07D9F90808EF30E7A5EAC39EF3
:200A400050A07420120B070A80F3B4630BAA01120AABE6120B0780DFB4732BC082C0838617
:200A6000820886837A00E4936004A30A80F88683188682120AABE493A36005120B0780F660
:200A8000D083D08280B1B4691986017A00E76004090A80F9120AAB8601E7609B120B070915
:200AA00080F7F97A01120AABE980A8EE601B8FF020F716C002EAC39E500D742030F60274C4
:200AC00030120B070A80EED0022278FB120B9C8603088604748075F070120C14120C687519
:200AE0008921F58DF58B7588597598522278FB120B9C8682088683E493602D120B07A380E3
:200B0000F678FB120B9CE63099FDC299F599B40A17740D80F2E430980C3098FDC298E59901
:200B2000B40D02740A75F0002278FB120B9CE63099FDC299F5992274FFF5F030980A309818
:200B4000FDC298E59975F0002278FB120B9C8601E4FBFCFFE709B42D030FE709C39430B49E
:200B60000A005012FA740A75F000120C002AFBE5F03400FC80E4EB8CF0DF03020C68227827
:200B8000FB120B9C8603088604BB0004BC00012279E5A3D9FD1BBBFFF01C80F4C82581C886
:200BA00022C92581C97A0022D083D082CF2581F581CFC082C08322CF2581F581CF2229F93B
:200BC000E5F03AFA227C00CB30E7011CCB2275F00030E70215F022FDE493A3FEE493A3FFAF
:200BE0004E7009E493FE740193FF800BE493A3B5050BE493B5F0068F838E82E473A380D8B2
:200C0000FEEBA4FD8EF0ECA4FCEB8EF0A4C5F02C2DC5F022C002C001AAF0F97E007D007FBE
:200C200011C3E933F9EA33FADF08F5F0E9D001D00222ED33FDEE33FEC3ED9BF5F0EE9C4004
:200C4000E0ADF0FED380DBBB000122C3C5F013C5F013DBF722120C5804700205F022120CA5
:200C60006114B4FF0215F022120C61F4C5F0F4C5F022120CC54029801E120CC5402270177A
:200C8000801E120CC540107017800C120CC550108005120CD96009E4F5F022120CD960F70F
:200CA000E4F5F00422120CD940F680EB120CD940EF70E480EB120CD940DD70E480D9120CE9
:200CC000D950DD80D2C39BC5F09C20E70720D207C345F02220D2F9D322C5F0C39C7003E5A0
:200CE000F09B22FBE493CB22FCE493FB740193CC22FAE493F9740193CA220A20456173796A
:200D00002D446F776E6C6F616465722056322E3120666F722041544D454C2038394335315C
:200D20002F35322F35355744000A203E000A206F6B000A2043484B53554D203D2025303482
:200D400078000A20666F756E6420383943253278002D313256002D3556000A206E6F6E62BD
:200D60006C616E6B202575206279746573000A20627974657320636F756E746572202575A1
:1C0D8000000A204E6F7420666F756E642038394378780025782C25752C257500D3
:00000001FF
